S02000006F70656E626C745F6F6C696D65785F73746D3332683130332E737265630F
S315080000000050002019040008010400080304000831
S315080000100504000807040008090400080000000099
S315080000200000000000000000000000000B040008AB
S315080000300D040008000000000F0400081104000861
S3150800004061040008610400086104000861040008EE
S3150800005061040008610400086104000861040008DE
S3150800006061040008610400086104000861040008CE
S3150800007061040008610400086104000861040008BE
S3150800008061040008610400086104000861040008AE
S31508000090610400086104000861040008610400089E
S315080000A0610400086104000861040008610400088E
S315080000B0610400086104000861040008610400087E
S315080000C0610400086104000861040008610400086E
S315080000D0610400086104000861040008610400085E
S315080000E061040008610400086104000800000000BB
S315080000F000000000000000000000000000000000F2
S3110800010000000000000000005FF808F195
S3150800010C10B5054C237833B9044B13B10448AFF337
S3150800011C00800123237010BDC800002000000000D9
S3150800012C3838000808B5034B1BB103490348AFF32D
S3150800013C008008BD00000000CC00002038380008FC
S3150800014C02F08EBF02F09BBF4FF40062024B0128EF
S3150800015C0CBF5A611A61704700100140704770470E
S3150800016C08B5054B9B68DB0703D500F037F801206B
S3150800017C08BD0020FCE700BF00080140642000F021
S3150800018C03B800F007B80000014B1880704700BF91
S3150800019CE400002010B502F075FD0C4C2268904264
S315080001AC0ED30B4B0B4A18784FF4805148B90120E3
S315080001BC1870516102F066FD074B1B8818442060C5
S315080001CC10BD002018701161F4E700BFE80000208C
S315080001DCE600002000100140E40000204FF4805295
S315080001EC014B1A61704700BF00100140054B82B0E5
S315080001FC9A6902439A619B6918400190019B02B067
S3150800020C704700BF00100240224B10B51A6822F046
S3150800021C070242F002021A601A6802F00702022A62
S3150800022CFAD11D4C236843F48033236023689A0360
S3150800023CFCD5636823F47C1343F4E81363602368E2
S3150800024C43F08073236023689B01FCD5636823F015
S3150800025CF0036360636823F4E06343F480636360CC
S3150800026C636823F460536360636823F0030343F005
S3150800027C02036360636803F00C03082BFAD1074882
S3150800028C01F07CFF002000F0F7F8636823F4800384
S3150800029C636010BD002002400010024000A24A0410
S315080002AC7FB500F00DF9FFF7AFFF1422002101A866
S315080002BC03F0B4FA2020FFF799FF0420FFF796FF06
S315080002CC1020FFF793FF4FF40063104C40F2011215
S315080002DC63614FF48053236104230D480DEB03012E
S315080002ECCDE9012301F01AF901230A490220CDE9C7
S315080002FC0113002301A9CDE90303204601F00EF9E9
S3150800030CFFF71EFFFFF71EFFFCE700BF00100140BA
S3150800031C0008014018001804104B82B09A6942F084
S3150800032C01029A619A6902F001020092009ADA694E
S3150800033C42F08052DA61DB69094A03F08053019373
S3150800034C019B536823F0E06343F080635360536862
S3150800035C23F0E063536002B0704700BF0010024000
S3150800036C000001400268084B82B09A420AD103F594
S3150800037CDA33DA6942F40002DA61DB6903F4000362
S3150800038C0193019B02B07047005C00400268044B65
S3150800039C9A4201BF034AD36923F40003D361704719
S315080003AC005C00400010024008B501F035F90E4813
S315080003BC01F064F80D4801F061F80D4BDA6922F486
S315080003CC0002DA619A6922F010029A619A6922F09F
S315080003DC04029A61DA6922F08052DA619A6922F08B
S315080003EC01029A6108BD00BF0010014000080140D7
S315080003FC001002407047FEE7FEE7FEE7FEE770478F
S3150800040C7047704700F06EB870470000002103E093
S3150800041C0B4B5B58435004310A480B4B42189A4213
S3150800042CF6D30A4A02E0002342F8043B084B9A42E8
S3150800043CF9D3FFF7E9FF03F0CDF9FFF731FF704762
S3150800044C0039000800000020C4000020C800002065
S3150800045CE80E0020FEE7000010B54FF0FF3200242E
S3150800046C044BDA601C61DA60DC60FFF79DFF2046FE
S3150800047C10BD00BF0010024038B50E4B0546187863
S3150800048C4FF47A73B3FBF0F30B4A1068B0FBF3F036
S3150800049C00F07AF8044658B90F2D09D802462946B1
S315080004AC4FF0FF3000F03CF82046044B1D6038BD79
S315080004BC0120FCE7040000200000002008000020B2
S315080004CC074A08B51368032043F01003136000F0BD
S315080004DC15F80020FFF7D0FFFFF71EFF002008BD18
S315080004EC00200240034A044B11681B780B44136026
S315080004FC704700BF840C002004000020074A000245
S3150800050CD36800F4E06023F4E0631B041B0C43F08F
S3150800051CBF6343F400330343D360704700ED00E038
S3150800052C174B70B5DC684FF0FF36C4F30224C4F1E0
S3150800053C0705042D04F1040328BF0425062B98BFD0
S3150800054C002406FA05F388BF033C21EA0303A340FB
S3150800055C06FA04F422EA0404002843EA0403A8BFB2
S3150800056C00F160404FEA0313B8BF064ADBB2ABBFD3
S3150800057C00F5614000F00F0080F80033135470BD8D
S3150800058C00ED00E014ED00E00138B0F1807F0AD2EE
S3150800059CF021064B064A586082F8231000200722E1
S315080005AC98601A6070470120704700BF10E000E0A1
S315080005BC00ED00E0114AD36813F0100305D010497A
S315080005CCCB6943F00203CB611023D268500706D5DA
S315080005DC0B4943F00403CA6942F00102CA61074A8F
S315080005ECD169C90708D50648C16941F00401C1613A
S315080005FCD16921F00101D161D36070470020024016
S3150800060C880C0020064B186910F0800007D0054AA4
S3150800061C5A6002F188325A601869C0F3C0107047E4
S3150800062C0020024023016745034A0020136943F062
S3150800063C80031361704700BF00200240F8B50646D8
S3150800064C02F028FB114C07462546E368D80712D456
S3150800065CE368990644BF2023E360EB68DA0606D400
S3150800066CEB69DB0703D4E86810F0040007D0FFF742
S3150800067CA1FF012003E0731CE7D00EB90320F8BDD7
S3150800068C02F008FBC01BB042DFD9F7E70020024096
S3150800069C2DE9F84F244C1E46237E0546012B0F46A2
S315080006AC90463FD001234CF250302376FFF7C6FF15
S315080006BCA0BB012D03D0022D0CBF022504254FF03B
S315080006CC0009CB46DFF864A04FEA0913C3F12001F1
S315080006DCA3F1200206FA01F128FA03F3C4F81CB0B8
S315080006EC0B4326FA02F21343DAF810209BB242F0B7
S315080006FC0102CAF810204CF2503027F81930FFF7CF
S3150800070C9DFFDAF8103023F00103CAF8103028B927
S3150800071C09F101095FFA89F39D42D5D8002323769E
S3150800072CBDE8F88F0220FBE7880C00200020024069
S3150800073C0022064BDA61064B1A6942F004021A616A
S3150800074C1A6942F040021A61704700BF880C0020F3
S3150800075C002002400022064BDA61064B1A6942F069
S3150800076C02021A6158611A6942F040021A6170470E
S3150800077C880C0020002002402DE9F041224D074646
S3150800078C2B7E8846012B3DD0012403682C76022B40
S3150800079C4CF2503013D1FFF751FF20B10120002342
S315080007AC2B76BDE8F081FFF7C3FF4CF25030FFF70C
S315080007BC45FF164A136923F004031361EFE7FFF7A5
S315080007CC3DFF0028EAD14FF0FF33C8F80030204629
S315080007DCBE680E4CD7E9023203EB8223B342DED94C
S315080007EC3046FFF7B7FF4CF25030FFF727FF236967
S315080007FC23F00203236110B1C8F80060CFE706F5B1
S3150800080C8066E7E70220CCE7880C0020002002402F
S3150800081CF0B5044687B010B390F8A93203F0FF027E
S3150800082C1BB980F8A822FFF79DFD254603236E46C3
S3150800083C55F8100B84F8A93200F02AFF0FCD0FC615
S3150800084C2B6825463360271D97E80E0055F8100BC4
S3150800085C00F00EFF064620B1022384F8A9320125C2
S3150800086C4BE00146206800F01DFF30464FF0010EA4
S3150800087C28260146D4F804C0C2B2944500F10100FA
S3150800088C18D8002328261946D8B2844503F1010343
S3150800089C1DD80FCD6E460FC62B68336097E80E0031
S315080008AC206800F001FF01230546F8B1022284F8FE
S315080008BCA922D4E706FB024383F829E083F828200B
S315080008CCDA8683F82B10C3E90E111964D4E706FBF4
S315080008DC004282F8691182F8680182F86B11C2F835
S315080008EC7811C2F87C11C2F88011CDE784F824007F
S315080008FC84F8A932206801F061F9284607B0F0BDE2
S3150800090C38B5044610B90125284638BD032380F8A6
S3150800091CA932006801F03FF905460028F3D12046B4
S3150800092CFFF734FD84F8A952EEE738B590F8A832EB
S3150800093C0446012B10D0012580F8A852006800F057
S3150800094C9EFE2946204602F03FFF206801F034F946
S3150800095C002084F8A80238BD0220FCE790F8A832DB
S3150800096C10B5012B044610D0012380F8A832006874
S3150800097C00F08EFE0021204602F026FF206801F0CA
S3150800098C1DF9002084F8A80210BD0220FCE790F897
S3150800099CA83210B5012B04460BD0012180F8A812F9
S315080009AC02F012FF206801F007F9002084F8A8026B
S315080009BC10BD0220FCE790F8A83210B5012B0446AE
S315080009CC0CD00123002180F8A83202F0FDFE206825
S315080009DC01F0F4F8002084F8A80210BD0220FCE708
S315080009EC90F8A82210B5012A04460BD0012280F8EB
S315080009FCA82284F82410006801F0D8F8002084F89E
S31508000A0CA80210BD0220FCE72DE9F04F044685B07C
S31508000A1C006801F0D5F8020409D5DFF82898DFF844
S31508000A2C28882068B0F844301B0400F1BC80206884
S31508000A3C01F0C6F843050FD522682046B2F84430B3
S31508000A4C23F480631B041B0CA2F8443002F0A9FDA6
S31508000A5C00212046FFF7C4FF206801F0B1F84704CF
S31508000A6C08D52268B2F8443023F480431B041B0CC7
S31508000A7CA2F84430206801F0A3F8860408D5226849
S31508000A8CB2F8443023F400531B041B0CA2F8443070
S31508000A9C206801F095F8C5041CD522682046B2F8E2
S31508000AAC403023F004031B041B0CA2F84030B2F8A8
S31508000ABC403023F008031B041B0CA2F8403002F04C
S31508000ACC8FFD2268B2F8443023F480531B041B0CA8
S31508000ADCA2F84430206801F073F8000541D50022CD
S31508000AEC236833F822102DF812100132082AF8D18F
S31508000AFCB3F8402042F00102A3F84020B3F8402096
S31508000B0C22F001021204120CA3F84020B3F8442078
S31508000B1C5105FBD5B3F8442022F480621204120C5A
S31508000B2CA3F8442000223DF8121023F822100132B3
S31508000B3C082AF8D1B3F84020204642F00802A3F858
S31508000B4C4020B3F8442022F400621204120CA3F8D5
S31508000B5C4420B3F8402042F00402A3F8402002F0E7
S31508000B6C2DFD206801F02CF882050BD5226820464D
S31508000B7CB2F8443023F400731B041B0CA2F844305F
S31508000B8C02F00BFD206801F01BF8C30508D5226896
S31508000B9CB2F8443023F480731B041B0CA2F84430BF
S31508000BAC05B0BDE8F08FB0F8441089B211F00F0605
S31508000BBC40F0B18011F0100103882AD109EA030329
S31508000BCC43F400430380B0F8503094F8282003EB24
S31508000BDCC20300EB4300B0F80434E26BC3F3090319
S31508000BEC63641344E363204602F0CFFC94F8243084
S31508000BFC002B3FF416AF226C002A7FF412AF94F840
S31508000C0C2430216843F08003A1F84C3084F8242062
S31508000C1C07E79BB213F4006520D0B0F8503094F86F
S31508000C2C682104F52C7103EBC20300EB4303B3F8FC
S31508000C3C0C34B4F86E21C3F30903C4F8843101F0FB
S31508000C4C81FA22682046138823F070031B051B0DB6
S31508000C5C43F08003138002F089FCE2E61F047FF55B
S31508000C6CE0AE038823F070031B051B0D43F08003CD
S31508000C7C0380B0F8503094F8682103EBC20300EBFC
S31508000C8C4303B3F80C34C3F30903C4F884318BB1AA
S31508000C9CD4F87C1171B1B4F86E2101F053FAD4F87A
S31508000CAC7C31D4F8842129461344C4F87C31204677
S31508000CBC02F062FC2168D4F87851B1F8503001F290
S31508000CCC0C409BB2BDB9C25A22F4F8421204120C5B
S31508000CDCC252C25A48EA020292B2C2520B8823F492
S31508000CEC804323F0700383F4405343F4004343F0EA
S31508000CFC80030B8095E63E2D05D86A08EE0748BF9B
S31508000D0C01329202E8E76A09ED0608BF02F1FF32E2
S31508000D1C48EA8222E0E730F82670BFB2390440F17F
S31508000D2CF280282130F8263001FB064123F07003A7
S31508000D3C1B051B0D43F0800320F8263091F87431FF
S31508000D4C00F5806CABB9B0F8503091F868210633D1
S31508000D5C03EBC2033CF81350C5F30905002D00F04C
S31508000D6CB6802B46B1F86E21D1F87C1101F0EAF960
S31508000D7CADE091F86B3191F86821022B40F089802F
S31508000D8C17F4804A4FEAC205D1F8803107F0400EB5
S31508000D9C3ED0B0F850A0554402353CF81550C5F372
S31508000DAC09059D428CBF00235B1BC1F880312823A3
S31508000DBC03FB0643D3F880316BB930F8223023F4A1
S31508000DCC804323F0700383F4005343F4004343F049
S31508000DDC800320F82230BEF1000F10D0282303FB25
S31508000DEC064393F8682130F8223023F0F0031B05EC
S31508000DFC1B0D43F4004343F0C00320F82230002DAA
S31508000E0C65D0282101FB06412B46B1F87021ABE7CA
S31508000E1CB0F850B05D4406353CF81550C5F30905D5
S31508000E2C9D429CBF5B1BC1F880314FF0280303FB26
S31508000E3C064388BFC1F880A1D3F880316BB930F866
S31508000E4C223023F4804323F0700383F4005343F4D5
S31508000E5C004343F0800320F82230BEF1000F10D176
S31508000E6C282303FB064393F8682130F8223023F035
S31508000E7CF0031B051B0D43F4004343F0C00320F895
S31508000E8C223025B3282101FB06412B46B1F87221E5
S31508000E9C6AE730F8223023F0F0031B051B0D43F4E8
S31508000EAC004343F0C00320F8223091F8683130F83B
S31508000EBC2320DB0012F4804FB0F850205ED00232AB
S31508000ECC13443CF81350C5F30905002D9CD1282171
S31508000EDC71436318D3F884212A44C3F88421D3F8C0
S31508000EEC7C212A44C3F87C21D3F880211AB1D3F883
S31508000EFC78319D424BD2282303FB0643204693F8B0
S31508000F0C681102F039FB3A067FF58BAD2825206867
S31508000F1C05FB064530F8263000F5806209EA03031E
S31508000F2C43F4004320F8263095F82B3095F8281012
S31508000F3C022B01D1FB053DD42823B0F850E003FB66
S31508000F4C064C0EF1020E0EEBC10132F81120DCF83C
S31508000F5C4070C2F30902974292BF0021BF1ACCF81F
S31508000F6C407003FB064798BFCCF84010396CA9B9FA
S31508000F7C95F82810204602F008FB52E50632134471
S31508000F8C3CF81350C5F30905002DA0D07DE701F5F3
S31508000F9CB4712144206800F029FEB4E7F96B06FB0E
S31508000FAC03331144F963796C0A447A64E11800F046
S31508000FBC1DFE36E517F0400E4FEAC10C2B6C07F4F4
S31508000FCC804700F09E80B0F850E0BFB2F4440CF1B4
S31508000FDC020C32F81CC0CCF3090C9C452CBF002320
S31508000FECA3EB0C032B64282303FB06431B6CABB93E
S31508000FFC204602F0CAFA002F00F0A18095F82810B6
S3150800100C226832F8213023F0F0031B051B0D43F43C
S3150800101C404343F0800322F8213090E05FB130F86A
S3150800102C213023F0F0031B051B0D43F4404343F01A
S3150800103C800320F82130282303FB064393F84C2021
S3150800104C012A7CD15A6CD96B62445A649F6C9A6B90
S3150800105C61449742D96325D3BF1A9F6495F82970C2
S3150800106C93B2002F41D1B0F8507000F2044CBC4436
S3150800107C95F828703F0102BB3CF8072022F4F84289
S3150800108C1204120C2CF807203CF8072048EA020236
S3150800109C92B22CF80720282202FB0646328E00F064
S315080010AC94FD4CE01FB983F84C706246D6E70022D3
S315080010BC83F84C209A643A46D0E73E2A0CD84FEA75
S315080010CC520ED20748BF0EF1010E4FEA8E2E1FFAAA
S315080010DC8EFE2CF807E0DEE74FEA521ED20608BF52
S315080010EC0EF1FF3E48EA8E2EF1E7012FD3D1B0F868
S315080010FC502000F20447174495F828201201BB52D9
S3150800110CC9E7B0F850A0BFB2D4440CF1060C32F8BB
S3150800111C1CC0CCF3090C9C459CBFA3EB0C032B649D
S3150800112C4FF0280303FB064388BFC5F840E01B6C49
S3150800113CBBB9204602F029FA002F3FF45FAF95F8A9
S3150800114C2810226832F8213023F4E04323F04003B8
S3150800115C83F0300343F4004343F0800322F8213034
S3150800116C5FE45FB930F8213023F0F0031B051B0D43
S3150800117C43F4404343F0800320F82130282303FB33
S3150800118C064393F84C20012AD9D15A6CD96B624480
S3150800119C5A649F6C9A6B61449742D96323D3BF1ADE
S315080011AC9F6495F8297093B2002F3FD1B0F8507010
S315080011BC00F20C4CBC4495F828703F01F2B93CF887
S315080011CC072022F4F8421204120C2CF807203CF8DB
S315080011DC072048EA020292B22CF80720282202FBC2
S315080011EC0646728E5BE71FB983F84C706246D8E7E1
S315080011FC00229A6483F84C203A46D2E73E2A0CD849
S3150800120C4FEA520ED20748BF0EF1010E4FEA8E2E48
S3150800121C1FFA8EFE2CF807E0E0E74FEA521ED206BC
S3150800122C08BF0EF1FF3E48EA8E2EF1E7012FD5D105
S3150800123CB0F8502000F20C47174495F828201201F4
S3150800124CBB52CBE70F8FFFFF0080FFFF11F0800F1B
S3150800125C70B501F0070504464FF028011CD005FBB4
S3150800126C01110144012048700A614A780D70CB704F
S3150800127C02B1CD81022B04BF00230B7194F8A8325E
S3150800128C012B13D00123206884F8A83200F020FA29
S3150800129C002084F8A80270BD002601FB05F000F5B5
S315080012ACB4712044214480F86961DDE70220F2E735
S315080012BC11F0800F10B501F0070204464FF0280113
S315080012CC13D0012302FB011101444B700A7094F8E8
S315080012DCA832012B13D00123206884F8A83200F019
S315080012EC35FB002084F8A80210BD01FB02F303F5B8
S315080012FCB47101440344002083F86901E6E702202F
S3150800130CF2E770B52824002601F007014C430519AD
S3150800131C85F8681104F5B4710144C5F87C21C5F843
S3150800132C8031C5F8846185F86961006800F05EFC57
S3150800133C304670BD282301F0070103FB0101D1F8E3
S3150800134C8401704770B5282501F0070105FB0104D7
S3150800135C0026C4E90F23012201FB055584F8281041
S3150800136C84F84C204119A364666484F82920006823
S3150800137C00F03CFC304670BD38B5436801F00705F3
S3150800138C9D42044628D811F0800F4FF028031AD036
S3150800139C05FB0333C11801234B7001230D708B70A9
S315080013AC94F8A8229A4219D084F8A832206800F03A
S315080013BC93FB25B904F52C71206800F004FC002079
S315080013CC84F8A80238BD00224B4303F5B4710344D4
S315080013DC014483F86921E0E70120F3E70220F1E7ED
S315080013EC38B5436801F00F029A42044626D811F024
S315080013FC800F01F007024FF0280115D0012302FBDC
S3150800140C011101444B7000250A708D7094F8A832AE
S3150800141C012B15D00123206884F8A83200F078FB3C
S3150800142C284684F8A85238BD01FB02F303F5B471BB
S3150800143C01440344002083F86901E4E70120F2E73C
S3150800144C0220F0E710B5282411F0800F1BBF01F01D
S3150800145C070101FB044104FB0100401808BF00F515
S3150800146CB47099B21AB90273C180002010BD01225A
S3150800147C1B0C027301814381F7E70000224B98424B
S3150800148C0BD103F58433DA6842F00402DA60DA68C1
S3150800149C22F00402DA60002070471C4B984209D1EE
S315080014AC03F58233DA6842F00802DA60DA6822F069
S315080014BC0802EFE7164B984209D103F58033DA6830
S315080014CC42F01002DA60DA6822F01002E2E7114BF9
S315080014DC984209D103F57C43DA6842F02002DA60B7
S315080014ECDA6822F02002D5E70B4B984209D103F5AE
S315080014FC7843DA6842F04002DA60DA6822F0400291
S3150800150CC8E70120704700BF00080140000C0140E5
S3150800151C0010014000140140001801402DE9F04F5D
S3150800152C0C68C4F30F2494FAA4F24FF00F0AB2FA1B
S3150800153C82F24FF0030904274FF0011C40F2011EFA
S3150800154C34FA02F302D11846BDE8F08F0123934012
S3150800155C23425ED0072A85BFA2F108030CFA03F3CF
S3150800156C0EFA02F343F08063C5681E0A96FAA6F8CB
S3150800157CB8FA88F825EA06060D6905FA08F535431A
S3150800158CC5604FEA136893FAA3F6B6FA86F693FA89
S3150800159CA3FBBBFA8BFBB6000AFA06F550F80860F3
S315080015AC4FEA8B0B26EA05064D6805FA0BFB46EA4D
S315080015BC0B0640F808604D6825F00805012D28D162
S315080015CC93FAA3F5B5FA85F593FAA3FBBBFA8BFB4D
S315080015DCAD0009FA05F526EA05068D684FEA8B0B68
S315080015EC05FA0BFB46EA0B0640F8086093FAA3F5D6
S315080015FCB5FA85F593FAA3F3B3FA83F3AD0007FAB4
S3150800160C05F526EA0505CE689B009E402E4340F854
S3150800161C0860013294E70000144B1A6842F0010284
S3150800162C1A601A689207FCD55A6822F003025A60A7
S3150800163C5A6812F00C0FFBD11A6822F080721A60E5
S3150800164C186810F00070FBD158601A6822F4502202
S3150800165C1A601A6822F0F80242F080021A60986042
S3150800166C5A6A42F080725A62704700BF00100240F4
S3150800167C84B001A880E80E0004B00020704700234F
S3150800168C4FF43F42A0F84430A0F840201846704763
S3150800169CB0F8403023F47C535B045B0CA0F8403064
S315080016AC002070470020704784B010B503AC84E85E
S315080016BC0E00BDE810400123A0F84030002304B00A
S315080016CCA0F84030A0F84430A0F8503018467047BF
S315080016DCF0B50C78034630F82420C87822F4EC428E
S315080016EC22F07002032803D8DFE800F0424944468A
S315080016FC012048F280052A4323F824200E78904AC4
S3150800170C33F82640354314402C4323F826400D7BEA
S3150800171C0C78002D40F08280CD884E786D086D00CF
S3150800172C03EB041476B3B3F850603444A4F80054AD
S3150800173C0D7833F82540670608D533F8254022403E
S3150800174C42F4004242F0C00223F82520CA780C78ED
S3150800175C012A33F824107B4A02EA010218BF82F0E8
S3150800176C200242F4004242F0800223F82420F0BD05
S3150800177C42F400720020BCE742F4C062FAE742F475
S3150800178C8062F7E7B3F850200E691444A4F808549D
S3150800179C0A78B3F8504003EB0212A4B202F20C42D8
S315080017AC56BB155B25F4F8452D042D0C1553155B06
S315080017BC45F4004515530C7833F8242057040BD5FB
S315080017CC33F8242022F0F0021205120D42F440429E
S315080017DC42F0800223F82420097833F8212022F4D9
S315080017EC804222F0700282F4405242F4004242F0E7
S315080017FC800223F82120BAE73E2E06D87508F6078C
S3150800180C48BF0135AD02ADB2D4E77709F5064E4DA2
S3150800181C08BF07F1FF3745EA8725F4E733F8245064
S3150800182C154045F4014545F0800523F824500C78FD
S3150800183C0D89B3F8506003EB04146D08B6B204F5C1
S3150800184C80646D00A5530C784D89B3F8506003EB92
S3150800185C04146D0804F581646D00B6B2A5534C7872
S3150800186C0D78B4BB33F82540660408D533F8254003
S3150800187C224042F4404242F0800223F825200C789C
S3150800188C33F8242055060BD533F8242022F0F00221
S3150800189C1205120D42F4004242F0C00223F824202D
S315080018AC48F280040D7833F8252022F4804222F081
S315080018BC700282F44052224323F82520097833F823
S315080018CC212022F4E04222F04002144323F821405E
S315080018DC4DE733F82540640408D533F825402240F3
S315080018EC42F4404242F0800223F825200C7833F863
S315080018FC242052060BD533F8242022F0F0021205C8
S3150800190C120D42F4004242F0C00223F82420CA7891
S3150800191C0C78012A33F824500A4A02EA050218BF41
S3150800192C82F0200242F4004242F0800223F824207E
S3150800193C097833F8212022F0F0029204920C54E72D
S3150800194C8F8FFFFFBF8FFFFF0080FFFF10B50C7B4B
S3150800195C4A780B78BCBBF2B130F8232052060BD56B
S3150800196C30F8232022F0F0021205120D42F4004240
S3150800197C42F0C00220F823200A7830F8223023F0EF
S3150800198CC0031B051B0D43F4004343F0800320F8EA
S3150800199C2230002010BD30F8232054040BD530F823
S315080019AC232022F0F0021205120D42F4404242F0B6
S315080019BC800220F823200A7830F8223023F0F0032E
S315080019CC9B049B0CDFE7002A44D130F823205204F1
S315080019DC0BD530F8232022F0F0021205120D42F432
S315080019EC404242F0800220F823200A7830F8223050
S315080019FC5C060BD530F8223023F0F0031B051B0DC3
S31508001A0C43F4004343F0C00320F822300A7830F838
S31508001A1C223023F0F0031B051B0D43F4004343F05F
S31508001A2CC00320F8223048F280020C7830F82430B3
S31508001A3C23F4804323F07003134320F824300978E9
S31508001A4C30F8213023F4E04323F040031A4320F8FE
S31508001A5C21209EE730F8232052040BD530F823209A
S31508001A6C22F0F0021205120D42F4404242F08002B6
S31508001A7C20F823200A7830F822305B060BD530F88C
S31508001A8C223023F0F0031B051B0D43F4004343F0EF
S31508001A9CC00320F822300A7830F8223023F0F003FD
S31508001AAC1B051B0D43F4404343F0800320F82230FA
S31508001ABC48F280020C7830F8243023F4E04323F003
S31508001ACC4003134320F82430097830F8213023F4E6
S31508001ADC804323F07003B9E74B780A787BB130F86A
S31508001AEC223023F4E04323F0400383F0100343F43D
S31508001AFC004343F0800320F822300020704730F86A
S31508001B0C223023F4804323F0700383F48053EEE7EA
S31508001B1C0B7B23BB4B780A781BB330F822305B0659
S31508001B2C0BD530F8223023F0F0031B051B0D43F4BC
S31508001B3C004343F0C00320F82230CB78012B0ED09B
S31508001B4C0A7830F8223023F4E04323F0400383F07C
S31508001B5C200343F4004343F0800320F8223000208E
S31508001B6C704730F822305B040BD530F8223023F05E
S31508001B7CF0031B051B0D43F4404343F0800320F888
S31508001B8C22300A7830F8223023F4804323F070038D
S31508001B9C83F44053DDE701220346A0F840200020D9
S31508001BAC0322A3F84400A3F84020704711B98023F8
S31508001BBCA0F84C3000207047002070470020704772
S31508001BCCB0F8440070470020704700EB420201331E
S31508001BDC02F580625B0802EB83039A4200D17047D8
S31508001BEC31F8020B22F8040BF7E70000F8B50C469F
S31508001BFC497805460129277B40F083812269A66925
S31508001C0C6169964228BF1646EFB9B6B23346E288E2
S31508001C1CFFF7DBFFB5F85010227805F204431201E2
S31508001C2C0B44D652227835F8223023F4E04323F0BD
S31508001C3C400383F03003002043F4004343F0800351
S31508001C4C25F82230F8BDE3782778022B40F024815A
S31508001C5C236A9A4230F8272022F4F8724FEA025285
S31508001C6C4FEA125280F0078142F4014242F0800298
S31508001C7C20F8272022789B1B30F82200236210F0CC
S31508001C8C400FB3B260787CD000284DD1B5F850001F
S31508001C9C05F20C4707441201002E31D1B85A20F42C
S31508001CACF8400004000CB852B85A40F40040B85238
S31508001CBC62892846FFF789FF226A236961699A4275
S31508001CCC89BF921B0023226232466078314498BF42
S31508001CDC2362616193B2002848D1B5F85000277881
S31508001CEC05F204463F01064442BBBA5B22F4F842AD
S31508001CFC1204120CBA53BA5B42F40042BA5326E0E9
S31508001D0C3E2E07D8700816F0010F18BF0130800256
S31508001D1C80B2CCE74FEA561CF006974808BF0CF180
S31508001D2CFF3C40EA8C20F3E70128C1D1B5F8507086
S31508001D3C05F20C40384412018352B9E73E2A0BD8F7
S31508001D4C5008D20748BF0130800280B2B8532289A6
S31508001D5C2846FFF73AFF65E75009D206864A08BFB8
S31508001D6C00F1FF3042EA802292B2C7E70128EED191
S31508001D7CB5F85060207805F20442000132448352CB
S31508001D8CE5E700284DD1B5F8500005F2044707449D
S31508001D9C1201002E31D1B85A20F4F8400004000C78
S31508001DACB852B85A40F40040B85222892846FFF770
S31508001DBC0CFF226A236961699A4289BF921B002328
S31508001DCC226232466078314498BF2362616193B2CD
S31508001DDC002845D1B5F85000277805F20C463F0186
S31508001DEC064442BBBA5B22F4F8421204120CBA53EC
S31508001DFCBA5B42F40042BA5326E03E2E07D8700866
S31508001E0C16F0010F18BF0130800280B2CCE74FEAFA
S31508001E1C561CF006584808BF0CF1FF3C40EA8C20CB
S31508001E2CF3E70128C1D1B5F8507005F204403844DF
S31508001E3C12018352B9E73E2A08D85008D20748BF80
S31508001E4C0130800280B2B853628981E75009D20604
S31508001E5C494A08BF00F1FF3042EA802292B2CAE72B
S31508001E6C0128F1D1B5F85060207805F20C42000132
S31508001E7C32448352E8E742F4004242F0800220F8EA
S31508001E8C2720B0F85070267800F204423A443601FE
S31508001E9C9BB2B35222895CE730F82720B0F8500081
S31508001EAC52064BBF05F20C4205F2044212181218E0
S31508001EBCB3B24FEA07174BBFD353D3536289228960
S31508001ECC2846FFF782FE6378227863B935F8223004
S31508001EDC23F0F0031B051B0D43F4004343F0C0032A
S31508001EEC25F822309EE6012B7FF49CAE35F822307D
S31508001EFC23F0F0031B051B0D43F4404343F080030A
S31508001F0CEEE7002F3AD1A269236905F20C419A42F1
S31508001F1C92BF1346D21AA261B0F85020207898BF07
S31508001F2CA7610001114453B9435A23F4F8431B041F
S31508001F3C1B0C4352435A43F40043435208E03E2BCE
S31508001F4C10D85A08DF0748BF0132920292B24252A1
S31508001F5C227835F8223023F4804323F0700383F477
S31508001F6C405368E65A09DE06034B08BF02F1FF32F6
S31508001F7C43EA82239BB2E0E70080FFFFE378022B5B
S31508001F8C74D199B9B0F8503000F20442217820691E
S31508001F9C09011A4400283AD18B5A23F4F8431B0436
S31508001FAC1B0C8B528B5A43F400438B526278237862
S31508001FBC002A50D1B5F85020206905F20C4111447D
S31508001FCC1B01002835D1CA5A22F4F8421204120C05
S31508001FDCCA52CA5A42F40042CA52E369002BB7D015
S31508001FEC44F24001227835F822300B408B4201D05E
S31508001FFC002BADD135F8223023F0F0031B051B0D51
S3150800200C43F4004343F0C00325F82230A0E73E28EA
S3150800201C06D84308C00748BF01339B029BB2C4E7E6
S3150800202C4609C706464B08BF06F1FF3643EA862320
S3150800203CF4E73E2806D84208C00748BF0132920288
S3150800204C92B2C9E74609C7063D4A08BF06F1FF36EC
S3150800205C42EA8622F4E7012ABFD1B5F8501005F2F8
S3150800206C0C420A44218A1B01D152B6E7012B64D1D2
S3150800207CA26923699A4295BF0023D21AA361A26169
S3150800208C98BF134689B9B0F85020207805F2044158
S3150800209C00011144FBB9425A22F4F8421204120CFC
S315080020AC4252425A42F4004242526178227800293E
S315080020BC37D1B5F8501005F20C4008441201E3B9B3
S315080020CC835A23F4F8431B041B0C8352835A43F498
S315080020DC004383523CE73E2B06D85A08DE0748BF16
S315080020EC0132920292B2DFE75E09DF06144A08BF94
S315080020FC06F1FF3642EA8622F4E73E2B07D8590842
S3150800210CDE0748BF0131890289B2815220E7590995
S3150800211CDB060B4B08BF01F1FF3143EA81239BB267
S3150800212CD7E701297FF414AFB5F8500005F20C4136
S3150800213C014412019BB28B520AE7012082E500BFCB
S3150800214C0080FFFF00EB4202F0B502F580625D08E5
S3150800215C084617462E46023036B9DB0744BF32F816
S3150800216C253001F81530F0BD37F8044B013EA4B202
S3150800217C00F8024C240A00F8014CECE7014B1860F5
S3150800218C704700BF0000002008B580B1D0F8B43203
S3150800219C13B10023C0F8B43209B1C0F8B012012348
S315080021AC027080F89C3201F025FA002008BD022046
S315080021BCFCE7012310B5044680F89C32D0F8B432FB
S315080021CC01795B689847204601F076FA204601F0BB
S315080021DC57FA002010BD19B1C0F8B4120020704788
S315080021EC0220704708B501F059FA002008BD08B559
S315080021FCD0F8B4320BB9022008BD1B6898470028E2
S3150800220CFAD0F8E708B5D0F8B4325B6898470020DE
S3150800221C08BD38B500F52A750446284600F0E2FADA
S3150800222C012394F8A812C4F89432B4F8AE32C4F860
S3150800223C983201F01F03012B0ED007D3022B10D0B6
S3150800224C01F08001204601F063FA03E02946204696
S3150800225C00F0F6F8002038BD2946204600F014FA9E
S3150800226CF8E72946204600F034FAF3E770B5054638
S3150800227C164649BBD0F89432032B1ED1D0F86031E0
S3150800228CD0F8642193420BD99B1A9A42C0F8603154
S3150800229C8CBF9AB292B2314600F0F4FA002070BDA7
S315080022ACD0F8B4321B6923B190F89C22032A00D1CA
S315080022BC9847284600F0EEFAF0E7052BEED1C5F85C
S315080022CC941201F025FAE9E7D0F8B4329B692BB1E0
S315080022DC90F89C22032A01D19847DFE70220DEE713
S315080022EC70B5134604460E46002947D1D0F89422F9
S315080022FC022A3CD1D0E90852954213D9AA1A02628D
S3150800230C194692B200F0B6FA33461A4619462046D2
S3150800231C01F048FA94F8A0320020012B01D184F878
S3150800232CA00270BDC369B3FBF2F502FB153565B99E
S3150800233C9A420AD8D0F89822934206D22A4600F036
S3150800234C99FAC4F898522B46DFE7D4F8B432DB680E
S3150800235C2BB194F89C22032A01D120469847802158
S3150800236C204601F0D5F9204600F09FFAD2E732F064
S3150800237C0403CFD1802101F0CBF9CBE7D0F8B432E6
S3150800238C5B6933B190F89C22032A02D19847002046
S3150800239CC7E70220C5E7002270B50446012540268A
S315080023AC1146402301F096F933468021C4F858515A
S315080023BCC4F864610022204601F08CF90021D4F897
S315080023CCB832A561666284F89C52C4F894126160AE
S315080023DCC4F8A41223B1D4F8B43220465B689847E3
S315080023EC002070BD01740020704790F89C3280F86C
S315080023FC9D32042380F89C320020704790F89C325A
S3150800240C042B04BF90F89D3280F89C32002070474C
S3150800241C08B590F89C22032A04D1D0F8B432DB69AB
S3150800242C03B19847002008BD10B50446802101F079
S3150800243C6FF92046BDE81040002101F069B900008B
S3150800244C37B50B78044603F06003202B0D4612D0E3
S3150800245C402B10D0002B5BD14B78092B58D8DFE8D2
S3150800246C13F0E90005015700FE005700840013001D
S3150800247C5700D200A000D4F8B43229469B682046EF
S3150800248C9847002003B030BD0023ADF806304B88C2
S3150800249C1A0A013A062A3BD8DFE802F004202D3A3C
S315080024AC3A525C00D0F8B0321B680DF10601207C5C
S315080024BC9847BDF8062052B1EB8843B19A4228BF1B
S315080024CC1A4601462046ADF8062000F0C6F9EB88F8
S315080024DC002BD6D1204600F0DDF9D2E7027CD0F8E5
S315080024ECB43232B99B6A0DF1060098470223437041
S315080024FCDFE7DB6AF7E7DBB2052B09D8DFE803F081
S3150800250C030C1014181CD0F8B0325B68002BCCD115
S3150800251C2046FFF789FFB4E7D0F8B0329B68F5E799
S3150800252CD0F8B032DB68F1E7D0F8B0321B69EDE7CA
S3150800253CD0F8B0325B69E9E7D0F8B0329B69E5E7C9
S3150800254C037C002BE4D1D0F8B4320DF106005B6B9A
S3150800255C9847AEE7037C002BDAD1D0F8B4320DF1EC
S3150800256C06001B6B98470723C1E78B88002BCFD136
S3150800257CCB88002BCCD14D887F2DC9D890F89C32AE
S3150800258C032BC5D0E9B280F89E1201F0EFF820466D
S3150800259C00F080F91DB1022384F89C3271E70123FF
S315080025ACFAE78978374D01292970B1D890F89C3209
S315080025BC022B08D0032B14D0FFF736FF29782046B8
S315080025CCFFF720FE5DE7002984D001210323416033
S315080025DC80F89C322046FFF70AFE02287FF47AAF71
S315080025EC96E731B90223416080F89C32FFF70AFE60
S315080025FC70E7416801293FF46DAFC9B2FFF702FED7
S3150800260C29786160E6E7CA88012A81D190F89C325C
S3150800261C002B3FF47DAF022B04D9032B7FF478AF44
S3150800262C011D03E00146002341F8083F204600F04F
S3150800263C14F926E790F89C32013B022B3FF668AF5B
S3150800264CCB88022B7FF464AF0123C360D0F8A43285
S3150800265C0BB10323C360022204F10C01E6E74B8895
S3150800266C012B7FF40EAFC4F8A43233E790F89C32F2
S3150800267C013B022B3FF64CAF4B88012B7FF401AF85
S3150800268C0023F0E7EC00002038B50B78044603F07D
S3150800269C6003202B0D4602D0402B00D0ABB994F822
S315080026AC9C32013B022B10D82B79012B0DD8D4F870
S315080026BCB43229469B6820469847EB881BB910B953
S315080026CC204600F0E7F8002038BD2046FFF7ACFEA0
S315080026DCF9E738B50A78044602F06002202A0B4658
S315080026EC14D0402A12D06AB95A788D88012AE9B2D0
S315080026FC20D036D3032A05D190F89C22022A27D05B
S3150800270C032A0BD02046FFF78FFE05E0D4F8B42237
S3150800271C1946926820469047002038BD5A882AB92F
S3150800272C4A0603D0DB880BB900F0F2FF204600F00E
S3150800273CB1F8F1E790F89C22022A09D0032AE1D1D4
S3150800274C5B88002BE8D14D06F0D000F0EFFFEDE7E3
S3150800275C4B06D7D000F0DCFF8021204600F0D8FFCE
S3150800276CDAE790F89C32022B18D0032BCAD1142323
S3150800277C01F00F0215F0800F03FB02021FD09269BD
S3150800278C002ABFD001F07F0505FB0335054411F07F
S3150800279C7F031FD12B60022229460CE04A06B1D1D1
S315080027AC2B064FF000034FF002024CBF00F1140148
S315080027BC00F5AA710B60204600F04FF8ACE7D2F88A
S315080027CC5821002A9ED001F07F0503FB050505F567
S315080027DCAA75DCE7204600F0B7FF08B10123D9E754
S315080027EC2860D8E70B7803704B784370CA788B78D7
S315080027FC03EB022343804A790B7903EB022383808C
S3150800280CCA798B7903EB0223C380704710B504464B
S3150800281C802100F07DFF2046BDE81040002100F025
S3150800282C77BF30B588B105462B1A15F8014BDBB2C4
S3150800283C002CF9D101335B0013800B7003234B700A
S3150800284C0223013810F8015F05B930BD5A1CCD5466
S3150800285CD2B20233DBB28C54F4E71346022210B51B
S3150800286CC0F89422C0E907330A46002100F08CFF11
S3150800287C002010BD08B513460A46002100F084FF57
S3150800288C002008BD08B513460A46002100F08AFF49
S3150800289C002008BD08B50423C0F8943200231A4654
S315080028AC194600F071FF002008BD08B50523C0F8CD
S315080028BC943200231A46194600F074FF002008BD0E
S315080028CC72B6704762B67047FFF7FABF10B500F0DC
S315080028DCA1F9C8B1FDF744FCB0B100F0FFFBFDF758
S315080028ECBBFD00F0A5F900F097F9084B20F0604005
S315080028FC20F07F00986000F08FF94468FFF7E2FF3C
S3150800290C2346BDE81040184710BD00BF00ED00E097
S3150800291CF8B514464FF6FF75461A013CA4B2AC42FC
S3150800292C00D1F8BD0B784F1C8B5500F0FEFB3946D1
S3150800293CF3E72DE9F84305460024FDF763FE05F198
S3150800294C04082F6858F8046004EB070900F0EDFB3F
S3150800295C3246002349460220FDF79AFE60B9E35930
S3150800296CB3420BD10434B4F5007FEAD10124FDF748
S3150800297C5BFE2046BDE8F8830024F8E70446F6E734
S3150800298C38B50E4B044698420D4607D00C4A914270
S3150800299C12D0FFF7CEFF10B904460BE0094C23689A
S315080029AC9D4207D020464FF4007240F8045B294636
S315080029BCFFF7AEFF204638BD1C46F0E7F4020020B0
S315080029CC00400008F00000202DE9F0419846036805
S315080029DC21F4FF76013304460D46174626F0010608
S315080029EC06D140F8046B4FF400723146FFF790FF9E
S315080029FC2368B34205D020463146FFF7C1FF04468B
S31508002A0CE8B123680435ED1A254406F50076B84472
S31508002A1C00F08BFB231DEB1AB3F5007F06D320467B
S31508002A2C3146FFF7ADFF044648B1051D17F8013BC3
S31508002A3C474505F8013BEBD10120BDE8F0810020A4
S31508002A4CFBE700004FF0FF33024A1360024A13609B
S31508002A5C704700BFF0000020F402002030B40E4C82
S31508002A6C4D1E0B46211A8D4213D80C49884210D993
S31508002A7C411E1944A1420CD820F4FF71084C21F0D0
S31508002A8C0101A142014630BC0CBF06480648FFF7B7
S31508002A9C9BBF002030BC7047FFFF0108FF3F0008B2
S31508002AAC00400008F4020020F000002030B5002495
S31508002ABC1C4D4A1E2B1A87B09A42019420D820F432
S31508002ACC7F73194A23F00303934219D9421E0A4409
S31508002ADCAA4215D80144C91AC1F38F25C1F30901B5
S31508002AEC09B10135ADB20024049301230294059370
S31508002AFCFDF788FDA3B2AB4205D30124FDF794FD7F
S31508002B0C204607B030BD00F010FB01A902A8FDF75E
S31508002B1C33FE013420B9049B03F580630493E9E77B
S31508002B2C0024EBE7FFFF0108FF3F000807B50F4A33
S31508002B3C1368013317D0D2E901310B44D1680C481C
S31508002B4C0B4411690B4451690B449169D2690B44C6
S31508002B5C13445B4202AA42F8043D0421FFF77EFFA8
S31508002B6C03B05DF804FB0120FAE700BFF40200206D
S31508002B7C0C4100080D4B0E4A1B68126813440D4A8B
S31508002B8C126813440C4A126813440C4A126813440C
S31508002B9C0B4A126813440B4A126813440A4A126801
S31508002BACD3420CBF01200020704700BF004000082C
S31508002BBC04400008084000080C40000810400008B3
S31508002BCC14400008184000080C4100080A4808B5CB
S31508002BDC0368013305D109480368013306D101207E
S31508002BEC08BDFFF7A6FE0028F5D1F9E7FFF7A1FE09
S31508002BFC003018BF0120F3E7F4020020F000002093
S31508002C0C0048704700400008FFF71CBFFFF726BFB7
S31508002C1CFFF74CBFFFF7AEBFFFF7F2BF08B5FFF7DC
S31508002C2C85FF18B1BDE80840FFF7D0BF08BD000006
S31508002C3C0022024B1A605A609A60704710E000E056
S31508002C4C08B5FFF7F5FF054B054A05215A60002222
S31508002C5C9A601960034B1A6008BD00BF10E000E0CB
S31508002C6C3F190100F8040020044B1B68DB0341BF25
S31508002C7C034A136801331360704700BF10E000E085
S31508002C8CF804002008B5FFF7EFFF014B186808BDDC
S31508002C9CF804002008B5FFF7E7FF014B186808BDD4
S31508002CACF8040020012838B504460D4604D94FF41B
S31508002CBCDE710E4800F088F9182060430C490B1891
S31508002CCC5C7C1A7C94420ED0DA6815705A7C5C6867
S31508002CDC01325A74DA680132A242DA6001D90A580A
S31508002CECDA60012000E0002038BD00BF503800082B
S31508002CFC3C050020012870B505460E4604D94FF44C
S31508002D0CEF710D4800F060F918226A430B4CA318B2
S31508002D1C587C80B1996809783170597C58680139A2
S31508002D2C59749968013181424FF0010088BFA25845
S31508002D3C996088BF9A6070BD503800083C05002021
S31508002D4C10B540241D4B1E4903F118025A61002286
S31508002D5C481CC3E902001C8218601C85081901244A
S31508002D6C0A70184958600A60174983F82A40481CA3
S31508002D7C0C70164CC3E90800986101F14000D86143
S31508002D8CDA629A7412492046FFF7FEF91149204671
S31508002D9CFFF721FA2046FFF725FAD4F8C002FDF70B
S31508002DACF6FD00F03DF9B0F5FA6F05D2BDE8104016
S31508002DBC4FF4FA6000F02EB910BD00BF3C05002098
S31508002DCC700500206C050020B1050020F4050020D4
S31508002DDC740000201000002010B5054CD4F8C00271
S31508002DECFDF7E9FD2046BDE81040FFF7E2B900BF44
S31508002DFCF40500203F292DE9F04107460C4603D976
S31508002E0CB521134800F0E0F8124D21462878FFF753
S31508002E1C49FF012803D0B9210D4800F0D5F83E46E4
S31508002E2CDFF82C80A4B2F31B9BB2A34201D3BDE8F6
S31508002E3CF08100F07AF916F8011B2878FFF732FFB3
S31508002E4C0128F0D0C221404600F0BEF8EBE700BFDF
S31508002E5C50380008700500202DE9F8431E4B1F4E0C
S31508002E6C8046D3F8C0020F46FDF7CEFD34781C4DCC
S31508002E7C1C4B8CB929461878FFF73CFF012803D060
S31508002E8C00242046BDE8F8832B78013B3E2BF7D867
S31508002E9C154B30701C70F4E7DFF84C90187899F8DD
S31508002EAC001001312944FFF725FF01280446E7D114
S31508002EBC99F800302A780133DBB29A4289F8003047
S31508002ECCDED1691C4046FFF723FD0023337099F8C1
S31508002EDC00303B70D5E700BFF4050020F808002049
S31508002EECB8080020B1050020F90800202DE9F341A7
S31508002EFC184E3478012C04D94FF4FF71164800F09B
S31508002F0C63F81822154B02FB0434647CFCB1402C84
S31508002F1C28BF40240025DFF84080114F0DF107012A
S31508002F2C3078FFF7E7FE012804D04FF4A17140462C
S31508002F3C00F04AF89DF80730EB550135EBB29C4288
S31508002F4CECD82346064A8121064800F01DFC02B03F
S31508002F5CBDE8F08170050020503800083C050020BB
S31508002F6CFC040020F40500202DE9F041044600F08D
S31508002F7C7FFA05462146114800F022FC2C46104FD4
S31508002F8CDFF8408086B2631B9BB29E4209D800F0DC
S31508002F9C6FFABDE8F041024640230121074800F0CC
S31508002FAC01BC14F8011B3878FFF77CFE0128EAD01F
S31508002FBC4FF4B271404600F007F8E4E7F405002038
S31508002FCCB10500205038000808B500F0AEF8FCE74B
S31508002FDC10B500F0A1F8012814D00B4C2378012B5E
S31508002FEC10D1FFF74FFE094B094A1B6812681344A8
S31508002FFC03F5FA73984205D300232370BDE81040F5
S3150800300CFFF764BC10BD00BF00090020FC080020B7
S3150800301C04090020014B1860704700BFFC0800200B
S3150800302C014B1868704700BFFC08002008B5044B14
S3150800303C1B78012B03D1FFF725FE024B186008BD40
S3150800304C0009002004090020012208B5034B1A7058
S3150800305CFFF7ECFFBDE80840FFF7BABF00090020F0
S3150800306C08B5FFF731FC00F05EF8FFF7E9FDFFF74E
S3150800307CCBFD00F00FF8BDE80840FFF7E5BF08B533
S3150800308C00F053F8FFF7F0FD00F010F8BDE8084023
S3150800309CFFF79EBF08B500F055F8FFF751FE022260
S315080030AC014B1A7008BD00BF0C00002007B5094873
S315080030BC0DF10701FFF7D0FE012807D10222064BB6
S315080030CC9DF8071003481A7000F058F803B05DF81D
S315080030DC04FB00BF080900200C000020FFF77CBE8B
S315080030EC08B5054B1B78022B02D1C9B2FFF782FE35
S315080030FCBDE8084000F03AB80C000020044B1B78D9
S3150800310C012B03D9032B01D03F20704700207047B1
S3150800311C0C000020FFF7F2BF08B500F01FF80030CE
S3150800312C18BF012008BDFDF729B8FDF72AB800001D
S3150800313CFE22034BDA7002221871A3F8442070475A
S3150800314C480900200022044B9A6483F84220A3F80D
S3150800315C44201A809A70704748090020024B187848
S3150800316C003018BF01207047480900200022024B86
S3150800317C83F84220704700BF48090020F8B5037849
S3150800318C0546FF2B7D4C2CD1E370102301252371AA
S3150800319C002325806371FFF7B1FFA071FFF7BAFF13
S315080031ACE071FFF7B7FF0823000A20726572A57253
S315080031BCA4F84430FFF728FD94F84230012B02D1CD
S315080031CC1020FFF7B5FFB4F94410002940F3D4805A
S315080031DC012389B284F842306948BDE8F840FFF704
S315080031EC7FBF2678012E40F0C780F32B58D01FD806
S315080031FCCF2B00F0BE8007D8C92B00F08380CC2BD0
S3150800320C00F08980202030E0D12B00F0AB80C0F094
S3150800321C8C80D22BF6D10025FF232571E3706571BE
S3150800322CFFF76CFFE571A0712572657207232BE019
S3150800323CFA2B4CD00BD8F52B11D028D3F62BE1D181
S3150800324CFF23E3704368A364A4F84460B4E7FD2B3A
S3150800325C49D0FE2B51D0FC2BD4D1002005E0FFF72A
S3150800326C4DFF6A78904203D82220FFF761FFA3E747
S3150800327CA16C201DFFF74CFBFF23E3706A78A36C47
S3150800328C1344A3646B780133A4F8443094E7FFF72E
S3150800329C35FF6B788342E7D26968A1646A78E8E7F8
S315080032ACFF230025E370A66C47683744BE4207D156
S315080032BC0123A3800023C4F80750A3710823E3E76E
S315080032CC16F8013B1D44EDB2FFF72FFFEEE7FF237F
S315080032DCE3702C4BA364002323716371A37107233A
S315080032ECC4F80730EAE7FF23E370002362782371FA
S315080032FCE380237262710623C6E700232380FF232B
S3150800330CE370A1E7A76CFFF7F9FE6A1C411E384665
S3150800331CFFF77CFC08B93120A7E7FF23E370FFF71A
S3150800332CEDFEA36C013803448DE7FFF7E7FE6B78D7
S3150800333C0138984298DDFF23A4F84460E370697855
S3150800334C29B9FFF76BFC00287FF436AFE3E7AA1C14
S3150800335CA06CFFF75BFC0028DDD06A78A36C1344DD
S3150800336CA36429E74168A06CFFF752FC0028C6D174
S3150800337CD1E7FFF7ABFAC2E7F8BD00BF4809002052
S3150800338C4B0900208C38000820230380004870471E
S3150800339C480000200A230380004870476800002074
S315080033AC08B590F89C32032B01D1FFF79FFD00203E
S315080033BC08BD08B5FFF79AFD002008BD08B50846F4
S315080033CCFFF7D2FD002008BD10B50446812100F098
S315080033DC91F90121204600F08DF9002010BD00005E
S315080033EC10B5044640230222812100F073F94023CC
S315080033FC02220121204600F06DF94023034A0121DF
S3150800340C204600F0CFF9002010BD00BFA80C002004
S3150800341C10B50A78044612F0600F12D14A780A2AB7
S3150800342C14D00B2A15D0062A0BD14A88120A212A3F
S3150800343C09D1CA880B49172A28BF17222046FFF735
S3150800344C0CFA002010BD08491722F7E70122074994
S3150800345CF5E78B7813B9054A1360F2E7FFF7D6F947
S3150800346CEFE700BF5A000020510000209409002005
S3150800347C00487047A80C0020122301480B8070479F
S3150800348C90000020042301480B807047A4000020FC
S3150800349C002370B51E46050FECB2092D94BF3034C7
S315080034AC373401F8134001EB430401336670DCB280
S315080034BCA2424FEA0010EED870BD00001A2310B5D0
S315080034CC0B80094B186808331B68C0180AD0074BC1
S315080034DC08221C680649FFF7DBFF0422054920462B
S315080034ECFFF7D6FF044810BDE8F7FF1FECF7FF1FE0
S315080034FCAA000020BA000020A800002010B5044C31
S3150800350C0A4604482146FFF78CF9204610BD00BF31
S3150800351CE80C0020B238000810B5044C0A460448DA
S3150800352C2146FFF77EF9204610BD00BFE80C0020A7
S3150800353CBF38000810B5044C0A4604482146FFF764
S3150800354C70F9204610BD00BFE80C0020943800081E
S3150800355C10B5044C0A4604482146FFF762F9204682
S3150800356C10BD00BFE80C00209C38000800F52C7133
S3150800357CD0F8E802FEF74DBE282303FB0103D0F86A
S3150800358CE802D3F87C21FEF771BE282303FB01035E
S3150800359CD0F8E802DA6BFEF7A3BED0F8E802FEF71D
S315080035AC37BF10B504460121D0F8E802FEF71AFF1A
S315080035BCD4F8E802BDE81040FEF7EDBE10B5044697
S315080035CCFCF7CCFDD4F8E802FEF70FFFA36923B18C
S315080035DC024A136943F00603136110BD00ED00E0BF
S315080035EC08B5D0F8E802FEF709FFBDE80840FCF775
S315080035FCB6BD0000082310B51E4A04461E48C0E98D
S3150800360C0023022383600023C0F8E842C4F8C002F2
S3150800361CC0E906330362FDF7FBF820B14FF49F713E
S3150800362C1648FFF7D1FC002218231146D4F8C0021D
S3150800363CFDF708FF582300228021D4F8C002FDF7B5
S3150800364C01FFC02300228121D4F8C002FDF7FAFE3F
S3150800365C4FF4887300220121D4F8C002FDF7F2FE5C
S3150800366C4FF4807300228221D4F8C002FDF7EAFEDB
S3150800367C002010BD005C004098090020D6380008D0
S3150800368C08B5D0F8C002FDF73BF9032896BF024BE4
S3150800369C0220185C08BD00BFD238000808B5D0F85F
S315080036ACC002FDF742F9032896BF024B0220185CAC
S315080036BC08BD00BFD238000808B5D0F8C002FDF71F
S315080036CC4DF9032896BF024B0220185C08BD00BFB3
S315080036DCD238000810B51C46D0F8C002134622464C
S315080036ECFDF7B4FD032896BF014B0220185C10BDEC
S315080036FCD238000808B5D0F8C002FDF7D9FD032862
S3150800370C96BF024B0220185C08BD00BFD2380008D1
S3150800371C08B5D0F8C002FDF72FFE032896BF024B5A
S3150800372C0220185C08BD00BFD238000808B5D0F8CE
S3150800373CC002FDF755FE032896BF024B0220185C03
S3150800374C08BD00BFD2380008282211F0800FD0F827
S3150800375CC0021BBF01F07F0303FB022102FB010120
S3150800376C091814BF887891F86A01704708B5D0F81B
S3150800377CC002FDF735F9032896BF024B0220185CE8
S3150800378C08BD00BFD238000808B5D0F8C002FDF74E
S3150800379CD9FD032896BF024B0220185C08BD00BF52
S315080037ACD238000808B5D0F8C002FDF7AAFD0328E0
S315080037BC96BF024B0220185C08BD00BFD238000821
S315080037CCD0F8C002FDF7B6BD01290CBF084600208B
S315080037DCFCF7BABC70B500250C4E0D4CA41BA410F6
S315080037ECA54209D100F022F800250A4E0A4CA41B62
S315080037FCA410A54205D170BD56F825309847013559
S3150800380CEEE756F8253098470135F2E7F838000800
S3150800381CF8380008F8380008FC3800080346024453
S3150800382C934200D1704703F8011BF9E7F8B500BFBE
S3150800383CF8BC08BC9E467047F8B500BFF8BC08BC77
S3090800384C9E467047CF
S31508003850433A2F576F726B2F736F66747761726571
S315080038602F4F70656E424C542F5461726765742FE2
S31508003870536F757263652F41524D434D335F5354F1
S315080038804D333246312F7573622E63004F70656E65
S31508003890424C540044656661756C740057696E55F0
S315080038A053422042756C6B20496E7465726661637B
S315080038B065004F70656E424C54205573657200570B
S315080038C0696E5553422042756C6B20446576696370
S315080038D06500000201022E2E2F5553425F444556BD
S315080038E04943452F5461726765742F757362645F27
S30D080038F0636F6E662E6300008B
S309080038F83101000884
S309080038FC0D010008A4
S315080039000024F4000100000010000000040000007C
S31508003910ED330008D53300081D3400080000000008
S3150800392000000000BF330008C9330008AD330008A3
S3150800393000000000000000000000000095330008A9
S3150800394000000000A133000809022000010100C0A0
S31508003950320904000002FF0000000705810240004A
S31508003960FF070501024000FF0A061001000000409B
S315080039700100000085340008913400080935000864
S3150800398025350008C9340008413500085D350008AA
S315080039901201100100000040501DAC600001010238
S315080039A003010000040309041A03000000000000D4
S315080039B000000000000000000000000000000000F9
S309080039C000000000F5
S70508000419D5
